:100000000C945E010C94FA1F0C94CF1F0C94A41F47
:100010000C94791F0C944E1F0C94231F0C94F81E03
:100020000C94CD1E0C9491010C9491010C949101AF
:100030000C9491010C9491010C9491010C949101F8
:100040000C9491010C9491010C9491010C949101E8
:100050000C9491010C9491010C9491010C94831EC9
:100060000C9491010C944F200C9425200C94910138
:100070000C9491010C9491010C9491010C948520A5
:100080000C9491010C9491010C9491010C949101A8
:100090000C9491010C9491010C9491010C94910198
:1000A0000C9491010C9491010C9491010C94910188
:1000B0000C9491010C9491010C9491010C94910178
:1000C0000C9491010C9491010C9491010C94910168
:1000D0000C9491010C9491010C9491010C94910158
:1000E0000C9491010C9418030C949F020C94F81A30
:1000F0000C94A9020C94C3010C949E1B0C94FA025C
:100100000C94BB030C94C3020C940B020C94F002ED
:100110000C94CF030C94BB020C947E030C94FD0151
:100120000C946D1C0C94E2010C94D7020C94010207
:100130000C94321C0C9404030C94E9010C941504E7
:100140000C94B3020C9488020C9467040C949502EE
:100150000C9490020C94CD020C94DA010C94391B8F
:100160000C945F1B0C94DE010C94C8010C941502D6
:100170000C94AC030C94E1020C947F030C94DD030B
:100180000C94E6010C9419020C9422030C942F2178
:100190000C94F3010C94241C0C940E030C94EF01AA
:1001A0000C940F020C94831C0C94F9010C9407021C
:1001B0000C94381B00002100240027002A002D0089
:1001C0003000330001010000040107010A010000B2
:1001D0002200250028002B002E00310034000201EF
:1001E0000000050108010B010505050507050808C4
:1001F0000808020202020A0A0808040404040101B1
:1002000001010101010103030303030303030407C5
:1002100007070C0C0C0C0C0C0C0C0202020206065C
:100220000606060606060B0B0B0B0B0B0B0B01024F
:1002300010202008081020401020408002010201F8
:1002400008040201010204081020408080402010B0
:100250000804020180040201804020100804020109
:100260000804020101020408102040800102040871
:100270001020408000000A0B02090C0D0E08070335
:100280000401000000000000000000000000000069
:10029000000000000000000000000000000000005E
:1002A000121110000000000000000000000000001B
:1002B000000000000000000000002F212092211FFC
:1002C00011241FBECFEFD1E2DEBFCDBF00E00CBFD7
:1002D00012E0A0E0B2E0E6E1FEE500E00BBF02C004
:1002E00007900D92A83AB107D9F72FE1A8EAB2E03A
:1002F00001C01D92A132B207E1F711E0CEE5D1E0D5
:1003000000E006C021970109802FFE010E940C2DFC
:10031000CD35D10780E00807A9F70E9484210C940D
:10032000092F0C940000282F30E0F901EC58FD4F04
:100330009491F901E25DFD4F449128513E4FF9013E
:100340002491222309F435C0992311F1915092315F
:10035000F8F4E92FF0E08827EF54FE4F8F4F0C940C
:100360000C2DE201E601C301DA01DE01C801E90159
:10037000EF01F301F901FD01010207020B02C801BF
:100380000F0215021902809180008F778093800000
:10039000E22FF0E0EE0FFF1FE253FE4FA591B49164
:1003A0008FB7F894EC91611148C040954E234C935F
:1003B0008FBF0895809180008F7DE8CF809180006D
:1003C000877FE4CF84B58F7784BDE2CF84B58F7DFE
:1003D000FBCF8091B0008F778093B000D9CF809110
:1003E000B0008F7DF9CF809190008F77809390003F
:1003F000CFCF809190008F7DF9CF80919000877F43
:10040000F5CF8091A0008F778093A000C1CF80911D
:10041000A0008F7DF9CF8091A000877FF5CF8091DC
:1004200020018F7780932001B3CF809120018F7DB1
:10043000F9CF80912001877FF5CF4E2BB8CFCF9396
:10044000DF9390E0FC01E25DFD4F249188519E4FC7
:10045000FC0184918823D1F090E0880F991FFC0162
:10046000EC54FE4FA591B491FC01E253FE4FC591AF
:10047000D49161110EC09FB7F8948C91E22FE09552
:100480008E238C932881E223E8839FBFDF91CF9155
:1004900008958FB7F894EC91E22BEC938FBFF6CFD1
:1004A0001F93CF93DF93182FEB0161E00E941F028F
:1004B000209739F460E0812FDF91CF911F910C9448
:1004C0009301CF3FD10511F461E0F5CFE12FF0E0CA
:1004D000EC58FD4FE491E150E23108F0B3C0F0E098
:1004E0008827EA58FD4F8F4F0C940C2D88029002FC
:1004F00095029F02A9022203B302BB02C302CD02EE
:10050000D702E102F002FA02220304030E031803E9
:1005100084B5806884BDC7BDDF91CF911F910895D8
:1005200084B5806284BDC8BDF7CF809180008068AB
:1005300080938000D0938900C0938800EDCF809194
:100540008000806280938000D0938B00C0938A00EB
:10055000E3CF80918000886080938000D0938D00ED
:10056000C0938C00D9CF8091B00080688093B00098
:10057000C093B300D1CF8091B00080628093B0006F
:10058000C093B400C9CF80919000806880939000A0
:10059000D0939900C0939800BFCF80919000806263
:1005A00080939000D0939B00C0939A00B5CF809128
:1005B0009000886080939000D0939D00C0939C0031
:1005C000ABCF8091A00080688093A0008091A000B4
:1005D0008F7B8093A000D093A900C093A8009CCFEC
:1005E0008091A00080628093A000D093AB00C09364
:1005F000AA0092CF8091A00088608093A000D09341
:10060000AD00C093AC0088CF8091200180688093BA
:100610002001D0932901C09328017ECF8091200131
:10062000806280932001D0932B01C0932A0174CF64
:1006300080912001886080932001D0932D01C09388
:100640002C016ACFC038D1050CF03ECF33CF3FB775
:10065000F89480915D1E90915E1EA0915F1EB091F6
:10066000601E26B5A89B05C02F3F19F00196A11D5D
:10067000B11D3FBFBA2FA92F982F8827BC01CD01EC
:10068000620F711D811D911D42E0660F771F881F4B
:10069000991F4A95D1F708958F929F92AF92BF927A
:1006A000CF92DF92EF92FF924B015C010E942703F1
:1006B0006B017C010E9427036C197D098E099F093B
:1006C000683E734081059105A8F321E0821A9108E4
:1006D000A108B10888EEC80E83E0D81EE11CF11C09
:1006E00081149104A104B10429F7FF90EF90DF90E9
:1006F000CF90BF90AF909F908F9008950895AF9244
:10070000BF92CF92DF92EF92FF920F931F93CF93FE
:10071000DF936C017B018B01040F151FEB015E0160
:10072000AE18BF08C017D10759F06991D601ED91F5
:10073000FC910190F081E02DC6011995892B79F784
:10074000C501DF91CF911F910F91FF90EF90DF9046
:10075000CF90BF90AF900895FC01538D448D252F0D
:1007600030E0842F90E0821B930B541710F0CF964B
:10077000089501970895FC01918D828D981761F07D
:10078000A28DAE0FBF2FB11D5D968C91928D9F5F94
:100790009F73928F90E008958FEF9FEF0895FC0173
:1007A000918D828D981731F0828DE80FF11D858D26
:1007B00090E008958FEF9FEF0895FC01918D228DB9
:1007C000892F90E0805C9F4F821B91098F7399273E
:1007D000089581E69EE10E94DD0321E0892B09F462
:1007E00020E0822F0895FC01A48DA80FB92FB11D20
:1007F000A35ABF4F2C91848D90E001968F73992757
:10080000848FA689B7892C93A089B1898C91837034
:1008100080648C93938D848D981306C00288F3892D
:10082000E02D80818F7D80830895EF92FF920F935A
:100830001F93CF93DF93EC0181E0888F9B8D8C8D8C
:1008400098131AC0E889F989808185FF15C09FB780
:10085000F894EE89FF896083E889F9898081837043
:10086000806480839FBF81E090E0DF91CF911F91F2
:100870000F91FF90EF900895F62E0B8D10E00F5F13
:100880001F4F0F731127E02E8C8D8E110CC00FB6E9
:1008900007FCFACFE889F989808185FFF5CFCE0181
:1008A0000E94F303F1CFEB8DEC0FFD2FF11DE35A06
:1008B000FF4FF0829FB7F8940B8FEA89FB89808104
:1008C0008062CFCF682F81E69EE10C941504CF9310
:1008D000DF93EC01888D8823B9F0AA89BB89E88968
:1008E000F9898C9185FD03C0808186FD0DC00FB60E
:1008F00007FCF7CF8C9185FFF2CF808185FFEDCF8C
:10090000CE010E94F303E9CFDF91CF91089580E0FB
:1009100090E0892B29F00E94E90381110E940000D8
:1009200080E090E0892B49F080E090E0892B29F06D
:100930000E94000081110E94000080E090E0892B5D
:1009400049F080E090E0892B29F00E94000081119D
:100950000E94000080E090E0892B49F080E090E068
:10096000892B29F00E94000081110C940000089549
:100970008091270A9091280AA091290AB0912A0A09
:10098000892B8A2B8B2BE1F08091230A9091240AEA
:10099000A091250AB091260A892B8A2B8B2B81F0F6
:1009A00080911602909117028F3F910549F0809136
:1009B000210A9091220A892B19F0109213020895AE
:1009C00081E0809313020895CF93DF9380EC90E051
:1009D0000E94620490E080E00E946204CBE1D3E0D8
:1009E0002091AA023091AB02CE018B519340821725
:1009F0009307A8F46991603C51F48BED90E00E945C
:100A000062046CED81E69EE10E941504E9CF6B3D26
:100A1000C9F78BED90E00E9462046DEDF3CF80EC9E
:100A200090E00E9462041092AB021092AA02DF9141
:100A3000CF91089580EC90E00E94620483E090E002
:100A40000E9462046091160281E69EE10E941504F4
:100A500080EC90E00C94620480EC90E00E946204D0
:100A600085E090E00E9462046091140281E69EE1BC
:100A70000E94150480EC90E00C94620480EC90E0FD
:100A80000E94620484E090E00E9462046091210A66
:100A900081E69EE10E94150480EC90E00C946204D3
:100AA00080EC90E00E94620486E090E00E94620484
:100AB0008091571E90E00E94620480EC90E00C94BC
:100AC0006204CF93C82F80EC90E00E94620480E91A
:100AD00090E00E9462046C2F81E69EE10E94150462
:100AE00080EC90E0CF910C946204803C51F48BED4B
:100AF00090E00E9462048CED682F81E69EE10C94E8
:100B000015048B3DC9F78BED90E00E9462048DEDDA
:100B1000F3CF1F93CF93DF9380EC90E00E946204A9
:100B200081E090E00E946204C091270AD091280AD7
:100B30001091290A80912A0A0E947505812F0E942E
:100B400075058D2F0E9475058C2F0E94750580EC10
:100B500090E0DF91CF911F910C9462041F93CF938B
:100B6000DF9380EC90E00E94620482E090E00E94BB
:100B70006204C091230AD091240A1091250A809121
:100B8000260A0E947505812F0E9475058D2F0E94EF
:100B900075058C2F0E94750580EC90E0DF91CF9158
:100BA0001F910C94620480EC90E00E94620484E245
:100BB00090E00E9462048091A9020E94750580EC79
:100BC00090E00C946204CF93C0910102C35680EC74
:100BD00090E00E94620483E290E00E9462048C2F05
:100BE0000E94750580EC90E0CF910C94620460E067
:100BF0008DE00C94930161E08DE00C949301CF9310
:100C0000DF93EC0161E08DE00E9493010E94F70503
:100C100064E670E080E090E00E944C030E94FB05D7
:100C200064E670E080E090E00E944C03219771F749
:100C3000DF91CF910C94F70560E08CE00C94930168
:100C40000F931F93CF93DF938C01EC01892B11F449
:100C5000C1E0D0E00E941C0664E670E080E090E015
:100C60000E944C0361E08CE00E94930164E670E016
:100C700080E090E00E944C030115110559F3219783
:100C800049F7DF91CF911F910F910C941C060E94A0
:100C9000FB050E941C066AE070E080E090E00E9484
:100CA0004C0361E08CE00E9493010E94F70565E02F
:100CB00070E080E090E00E944C03E9CF0F931F9317
:100CC000CF93DF938C01EC01892B11F4C1E0D0E0CC
:100CD00061E08CE00E94930160E08DE00E9493014E
:100CE00064E670E080E090E00E944C0360E08CE0FD
:100CF0000E94930161E08DE00E94930164E670E040
:100D000080E090E00E944C030115110509F3219742
:100D1000F9F60E941C06DF91CF911F910F910C9460
:100D2000F7052F923F924F925F926F927F928F9230
:100D30009F92AF92BF92CF92DF92EF92FF920F936A
:100D40001F93CF93DF93CDB7DEB7C857D1090FB646
:100D5000F894DEBF0FBECDBFE9969FAF8EAFE99787
:100D60001A01DC0118960D911D912D913C911B9754
:100D700061960CAF1DAF2EAF3FAF61971C960D91E2
:100D80001D912D913C911F9709831A832B833C83DE
:100D900050960D911D912D913C9153970D831E837B
:100DA0002F83388754960D911D912D913C91579723
:100DB00009871A872B873C87E6966FAFE697E796F9
:100DC0007FAFE797A85ABF4F6396BFAFAEAF6397A9
:100DD000FC01E45AFF4F6596FFAFEEAF65978C01BB
:100DE000005A1F4F67961FAF0EAF67979C012C5993
:100DF0003F4F69963FAF2EAF699788599F4F6B96CB
:100E00009FAF8EAF6B97E996AEADBFADE997A45992
:100E1000BF4F6D96BFAFAEAF6D97E996EEADFFAD2C
:100E2000E997E059FF4F6F96FFAFEEAF6F97E996E6
:100E30000EAD1FADE9970C581F4FA1961FAF0EAF17
:100E4000A197E9962EAD3FADE99728583F4FA3965D
:100E50003FAF2EAFA397E9968EAD9FADE99784582B
:100E60009F4FA5969FAF8EAFA597E996AEADBFAD4C
:100E7000E997A058BF4FA796BFAFAEAFA797E99627
:100E8000EEADFFADE997EC57FF4FA996FFAFEEAF80
:100E9000A997E9960EAD1FADE99708571F4FAB967E
:100EA0001FAF0EAFAB97E9962EAD3FADE997245734
:100EB0003F4FAD963FAF2EAFAD97E9968EAD9FAD4C
:100EC000E99780579F4FAF969FAF8EAFAF97E99648
:100ED000AEADBFADE997AC56BF4FE196BFAFAEAF79
:100EE000E197E796AEADBFADE7970D911D912D91BE
:100EF0003C910D871E872F87388B6396EEADFFAD33
:100F00006397008311832283338361968CAD9DADFB
:100F1000AEADBFAD619788589B45A549B842800FDB
:100F2000911FA21FB31F4D815E816F817885098556
:100F30001A852B853C854027512762277327098115
:100F40001A812B813C81402351236223732309851D
:100F50001A852B853C854027512762277327840FEC
:100F6000951FA61FB71F8C019D0147E0000F111FA1
:100F7000221F331F4A95D1F7AC01BD01E9E17695F7
:100F8000679557954795EA95D1F7402B512B622BE2
:100F9000732B89819A81AB81BC81480F591F6A1FCD
:100FA0007B1FE796AEADBFADE79714960D911D91EF
:100FB0002D913C911797098B1A8B2B8B3C8B659647
:100FC000EEADFFAD6597008311832283338389855E
:100FD0009A85AB85BC858A5A9844A843B741800F4F
:100FE000911FA21FB31FC980DA80EB80FC800D81A6
:100FF0001E812F813885C026D126E226F326C42201
:10100000D522E622F722C026D126E226F3268C0D31
:101010009D1DAE1DBF1D8C019D01FCE0000F111F29
:10102000221F331FFA95D1F76C017D01A4E1F694DC
:10103000E794D794C794AA95D1F7C02AD12AE22A77
:10104000F32AC40ED51EE61EF71EE796AEADBFAD61
:10105000E79718968D919D910D90BC91A02D8D8B49
:101060009E8BAF8BB88F6796EEADFFAD6797808391
:101070009183A283B3838D819E81AF81B885855290
:101080009F48AF4DBB4D0D891E892F89388D800F2C
:10109000911FA21FB31F49805A806B807C80442619
:1010A0005526662677264C205D206E207F200981FC
:1010B0001A812B813C814026512662267326840D9D
:1010C000951DA61DB71D8C019D01EFE03695279556
:1010D00017950795EA95D1F72C013D01F1E1440CF4
:1010E000551C661C771CFA95D1F7402A512A622AB2
:1010F000732A4C0C5D1C6E1C7F1CE796AEADBFAD19
:10110000E7971C968D919D910D90BC91A02D898F94
:101110009A8FAB8FBC8F6996EEADFFAD69978083D8
:101120009183A283B38389819A81AB81BC818251EF
:101130009143A244BE43098D1A8D2B8D3C8D800FA7
:10114000911FA21FB31F8A019B010C251D252E256F
:101150003F2504211521262137210427152726277D
:101160003727800F911FA21FB31F4C015D011AE0AA
:10117000B694A794979487941A95D1F78C019D0102
:1011800086E1000F111F221F331F8A95D1F708290E
:1011900019292A293B29040D151D261D371DE796FF
:1011A000AEADBFADE79750968D919D910D90BC91DE
:1011B000A02D8D8F9E8FAF8FB8A36B96EEADFFAD38
:1011C0006B9780839183A283B3838155904FA3480B
:1011D000BA40840F951FA61FB71FB701A60144256B
:1011E00055256625772540235123622373234C25FB
:1011F0005D256E257F25840F951FA61FB71F4C0107
:101200005D0147E0880C991CAA1CBB1C4A95D1F7CC
:10121000AC01BD01E9E17695679557954795EA954B
:10122000D1F7482959296A297B29400F511F621F8C
:10123000731FE796AEADBFADE79754968D919D9124
:101240000D90BC91A02D89A39AA3ABA3BCA36D96CE
:10125000EEADFFAD6D9780839183A283B383865DEE
:101260009943A847B84B8C0D9D1DAE1DBF1D730142
:101270006201C026D126E226F326C422D522E62228
:10128000F722C424D524E624F7248C0D9D1DAE1D21
:10129000BF1D4C015D01FCE0880C991CAA1CBB1C05
:1012A000FA95D1F76C017D01A4E1F694E794D79407
:1012B000C794AA95D1F7C828D928EA28FB28C40ED4
:1012C000D51EE61EF71EE796AEADBFADE797589662
:1012D0008D919D910D90BC91A02D8DA39EA3AFA348
:1012E000B8A76F96EEADFFAD6F9780839183A28311
:1012F000B3838D5E994BAF4CB745840D951DA61DEC
:10130000B71D2801390144265526662677264C202C
:101310005D206E207F204026512662267326840D94
:10132000951DA61DB71D4C015D01EFE0B694A79475
:1013300097948794EA95D1F72C013D01F1E1440C93
:10134000551C661C771CFA95D1F7482859286A283D
:101350007B284C0C5D1C6E1C7F1CE796AEADBFADB0
:10136000E7975C968D919D910D90BC91A02D89A7DA
:101370009AA7ABA7BCA7A196EEADFFADA1978083BE
:101380009183A283B3838F5F9A46A94BB240800FAB
:10139000911FA21FB31F8A019B010C251D252E251D
:1013A0003F2504211521262137210427152726272B
:1013B0003727800F911FA21FB31F4C015D011AE058
:1013C000B694A794979487941A95D1F78C019D01B0
:1013D00086E1000F111F221F331F8A95D1F70829BC
:1013E00019292A293B29040D151D261D371DE796AD
:1013F000AEADBFADE79790968D919D910D90BC914C
:10140000A02D8DA79EA7AFA7B8ABA396EEADFFAD5D
:10141000A39780839183A283B38388529746AF4773
:10142000B649840F951FA61FB71FB701A601442513
:1014300055256625772540235123622373234C25A8
:101440005D256E257F25840F951FA61FB71F4C01B4
:101450005D0147E0880C991CAA1CBB1C4A95D1F77A
:10146000AC01BD01E9E17695679557954795EA95F9
:10147000D1F7482959296A297B29400F511F621F3A
:10148000731FE796AEADBFADE79794968D919D9192
:101490000D90BC91A02D89AB9AABABABBCABA59624
:1014A000EEADFFADA59780839183A283B383815571
:1014B0009840AB4BB4478C0D9D1DAE1DBF1D7301F5
:1014C0006201C026D126E226F326C422D522E622D6
:1014D000F722C424D524E624F7248C0D9D1DAE1DCF
:1014E000BF1D4C015D01FCE0880C991CAA1CBB1CB3
:1014F000FA95D1F76C017D01A4E1F694E794D794B5
:10150000C794AA95D1F7C828D928EA28FB28C40E81
:10151000D51EE61EF71EE796AEADBFADE7979896CF
:101520008D919D910D90BC91A02D8DAB9EABAFABDD
:10153000B8AFA796EEADFFADA79780839183A28346
:10154000B3838F54944AA109B109840D951DA61D3A
:10155000B71D2801390144265526662677264C20DA
:101560005D206E207F204026512662267326840D42
:10157000951DA61DB71D4C015D01EFE0B694A79423
:1015800097948794EA95D1F72C013D01F1E1440C41
:10159000551C661C771CFA95D1F7482859286A28EB
:1015A0007B284C0C5D1C6E1C7F1CE796AEADBFAD5E
:1015B000E7979C968D919D910D90BC91A02D89AF40
:1015C0009AAFABAFBCAFA996EEADFFADA997808344
:1015D0009183A283B38382549842A34AB647800F73
:1015E000911FA21FB31F8A019B010C251D252E25CB
:1015F0003F250421152126213721042715272627D9
:101600003727800F911FA21FB31F4C015D011AE005
:10161000B694A794979487941A95D1F78C019D015D
:1016200086E1000F111F221F331F8A95D1F7082969
:1016300019292A293B29040D151D261D371DE7965A
:10164000AEADBFADE797D0968D919D910D90BC91B9
:10165000A02D21968CAF9DAFAEAFBFAF2197AB96BB
:10166000EEADFFADAB9780839183A283B3834C0132
:101670005D01FEED8F1AFEEE9F0AFFE6AF0AF4E968
:10168000BF0A840E951EA61EB71EB701A6014425EB
:1016900055256625772540235123622373234C2546
:1016A0005D256E257F25480D591D6A1D7B1D4A014C
:1016B0005B0197E0880C991CAA1CBB1C9A95D1F77A
:1016C000E9E17695679557954795EA95D1F74829C9
:1016D00059296A297B29400F511F621F731FE79602
:1016E000AEADBFADE797D4968D919D910D90BC9115
:1016F000A02D25968CAF9DAFAEAFBFAF2597AD9611
:10170000EEADFFADAD9780839183A283B3834C018F
:101710005D01FDE68F1AFEE89F0AF7E6AF0AF2E0E8
:10172000BF0A8C0C9D1CAE1CBF1C73016201C0263D
:10173000D126E226F326C422D522E622F722C424AB
:10174000D524E624F724C80CD91CEA1CFB1C46014E
:101750005701FCE0880C991CAA1CBB1CFA95D1F718
:10176000A4E1F694E794D794C794AA95D1F7C82832
:10177000D928EA28FB28C40ED51EE61EF71EE796D8
:10178000AEADBFADE797D8968D919D910D90BC9170
:10179000A02D29968CAF9DAFAEAFBFAF2997AF9666
:1017A000EEADFFADAF9780839183A283B3834C01ED
:1017B0005D01F2E78F1AFCEB9F0AF6E8AF0AF9E544
:1017C000BF0A840C951CA61CB71C280139014426AD
:1017D0005526662677264C205D206E207F204026E9
:1017E000512662267326480C591C6A1C7B1C530127
:1017F0004201BFE0B694A79497948794BA95D1F725
:1018000081E1440C551C661C771C8A95D1F7482849
:1018100059286A287B284C0C5D1C6E1C7F1CE7969F
:10182000AEADBFADE797DC968D919D910D90BC91CB
:10183000A02D2D968CAF9DAFAEAFBFAF2D97E1968B
:10184000EEADFFADE19780839183A283B3834C011A
:101850005D01FFED8F1AF7EF9F0AFBE4AF0AF6EB8D
:10186000BF0A800E911EA21EB31E8A019B010C2589
:101870001D252E253F25042115212621372104274A
:10188000152726273727080D191D2A1D3B1D48013E
:1018900059019AE0B694A794979487949A95D1F7B2
:1018A000E6E1000F111F221F331FEA95D1F7082927
:1018B00019292A293B29040D151D261D371D898844
:1018C0009A88AB88BC888EE9881A8AED980A81EEDE
:1018D000A80A89E0B80A840E951EA61EB71EB30199
:1018E000A20140275127622773274C215D216E21D9
:1018F0007F214425552566257725480D591D6A1DEC
:101900007B1D4A015B01F5E0880C991CAA1CBB1CDD
:10191000FA95D1F7ABE17695679557954795AA95D6
:10192000D1F7482959296A297B29400F511F621F85
:10193000731F8DA09EA0AFA0B8A490EC891A9CE460
:10194000990A9FEBA90A9FE3B90A8C0C9D1CAE1C57
:10195000BF1C68017901C426D526E626F726C420D7
:10196000D520E620F720C026D126E226F326C80C93
:10197000D91CEA1CFB1C46015701B9E0880C991CD4
:10198000AA1CBB1CBA95D1F787E1F694E794D794CB
:10199000C7948A95D1F7C828D928EA28FB28C40E0D
:1019A000D51EE61EF71E89AC9AACABACBCACAFEA58
:1019B0008A1AA5EA9A0AA1EAAA0AA9EDBA0A840C27
:1019C000951CA61CB71C2A013B014C245D246E24E7
:1019D0007F24402251226222732244265526662605
:1019E0007726480C591C6A1C7B1C530142019EE05F
:1019F000880C991CAA1CBB1C9A95D1F7E2E176943D
:101A0000679457944794EA95D1F7482859286A284B
:101A10007B284C0C5D1C6E1C7F1C8D849E84AF84C7
:101A2000B888B6E58B1AB8E39B0AB9E4AB0AB6E10D
:101A3000BB0A800E911EA21EB31E970186010425CB
:101A400015252625372504231523262337230C2582
:101A50001D252E253F25080D191D2A1D3B1D48015A
:101A60005901FCE0B694A79497948794FA95D1F71E
:101A7000A4E1000F111F221F331FAA95D1F70829D7
:101A800019292A293B29040D151D261D371D89A05A
:101A90009AA0ABA0BCA0E3EA8E1AEFEE9E0AE0ED9E
:101AA000AE0AE9E2BE0A840E951EA61EB71EB30159
:101AB000A20140275127622773274C215D216E2107
:101AC0007F214425552566257725480D591D6A1D1A
:101AD0007B1D4A015B01B5E0880C991CAA1CBB1C4C
:101AE000BA95D1F78BE176956795579547958A9585
:101AF000D1F7482959296A297B29400F511F621FB4
:101B0000731F8DA89EA8AFA8B8ACFDEA8F1AFBEE94
:101B10009F0AFBEBAF0AFDEFBF0A8C0C9D1CAE1CAD
:101B2000BF1C68017901C426D526E626F726C42005
:101B3000D520E620F720C026D126E226F326C80CC1
:101B4000D91CEA1CFB1C4601570199E0880C991C22
:101B5000AA1CBB1C9A95D1F7E7E1F694E794D794B9
:101B6000C794EA95D1F7C828D928EA28FB28C40EDB
:101B7000D51EE61EF71E2D968CAC9DACAEACBFAC50
:101B80002D978FE7881A89E1980A8EE5A80A87E2DF
:101B9000B80A840C951CA61CB71C2A013B014C24D6
:101BA0005D246E247F244022512262227322442627
:101BB000552666267726480C591C6A1C7B1C530147
:101BC0004201FEE0880C991CAA1CBB1CFA95D1F7B7
:101BD000A2E17694679457944794AA95D1F7482840
:101BE00059286A287B284C0C5D1C6E1C7F1C8D8C30
:101BF0009E8CAF8CB8A098E3891A94E0990A9CE275
:101C0000A90A98E1B90A800E911EA21EB31E97017F
:101C1000860104251525262537250423152326238B
:101C200037230C251D252E253F25080D191D2A1D9E
:101C30003B1D48015901BCE0B694A7949794879442
:101C4000BA95D1F784E1000F111F221F331F8A9527
:101C5000D1F7082919292A293B29040D151D261D0C
:101C6000371D89A89AA8ABA8BCA8AAE18A1AA2E342
:101C70009A0AAEE1AA0AAEEDBA0A840E951EA61E15
:101C8000B71EB301A20140275127622773274C21B9
:101C90005D216E217F214425552566257725480D38
:101CA000591D6A1D7B1D4A015B0195E0880C991C3A
:101CB000AA1CBB1C9A95D1F7EBE1769567955795D1
:101CC0004795EA95D1F7482959296A297B29400F78
:101CD000511F621F731F29968CAC9DACAEACBFAC7C
:101CE0002997BAE28B1AB8EF9B0AB8ECAB0ABCE3AF
:101CF000BB0A8C0C9D1CAE1CBF1C68017901C4265C
:101D0000D526E626F726C420D520E620F720C026D3
:101D1000D126E226F326C80CD91CEA1CFB1C46017E
:101D20005701F9E0880C991CAA1CBB1CFA95D1F745
:101D3000A7E1F694E794D794C794AA95D1F7C82859
:101D4000D928EA28FB28C40ED51EE61EF71E898C6A
:101D50009A8CAB8CBC8CE9E78E1AE2EF9E0AEAE221
:101D6000AE0AEBE0BE0A840C951CA61CB71C2A0127
:101D70003B014C245D246E247F24402251226222A8
:101D800073224426552666267726480C591C6A1C61
:101D90007B1C53014201BEE0880C991CAA1CBB1C91
:101DA000BA95D1F782E176946794579447948A95CF
:101DB000D1F7482859286A287B284C0C5D1C6E1CDA
:101DC0007F1C8DA49EA4AFA4B8A8F3E18F1AFBEEEC
:101DD0009F0AF5EAAF0AFAEBBF0A800E911EA21E17
:101DE000B31E9701860104251525262537250423D2
:101DF0001523262337230C251D252E253F25080DC9
:101E0000191D2A1D3B1D480159019CE0B694A79459
:101E1000979487949A95D1F7E4E1000F111F221F40
:101E2000331FEA95D1F7082919292A293B29040DDE
:101E3000151D261D371D25968CAC9DACAEACBFACD8
:101E400025978BEF881A86E1980A8CE1A80A86E527
:101E5000B80A840E951EA61EB71EB301A201402724
:101E60005127622773274C215D216E217F21442554
:101E7000552566257725480D591D6A1D7B1D4A018C
:101E80005B01F5E0880C991CAA1CBB1CFA95D1F7E4
:101E9000ABE17695679557954795AA95D1F748296F
:101EA00059296A297B29400F511F621F731F8D8892
:101EB0009E88AF88B88C98E0891A9CE5990A90E1D1
:101EC000A90A93E0B90A8C0C9D1CAE1CBF1C6801CA
:101ED0007901C426D526E626F726C420D520E6209B
:101EE000F720C026D126E226F326C80CD91CEA1C0E
:101EF000FB1C46015701B9E0880C991CAA1CBB1CAD
:101F0000BA95D1F787E1F694E794D794C7948A9568
:101F1000D1F7C828D928EA28FB28C40ED51EE61E0A
:101F2000F71E89A49AA4ABA4BCA4A7E28A1AADEFB9
:101F30009A0AA0E9AA0AA8E9BA0A840C951CA61C68
:101F4000B71C2A013B014C245D246E247F244022CF
:101F50005122622273224426552666267726480C93
:101F6000591C6A1C7B1C530142019EE0880C991C81
:101F7000AA1CBB1C9A95D1F7E2E17694679457941A
:101F80004794EA95D1F7482859286A287B284C0CB1
:101F90005D1C6E1C7F1C4601570184249524A624D9
:101FA000B72421968CAD9DADAEADBFAD21978657C0
:101FB000934BA54DB247800F911FA21FB31F9501F0
:101FC000840104231523262337230C251D252E25C4
:101FD0003F25800F911FA21FB31F8C019D01FCE0C4
:101FE0003695279517950795FA95D1F7E5960CAF95
:101FF0001DAF2EAF3FAFE5978C019D01A4E1000F0F
:10200000111F221F331FAA95D1F7E5968CAD9DAD08
:10201000AEADBFADE597082B192B2A2B3B2B040D3A
:10202000151D261D371D89A19AA1ABA1BCA18E5BF0
:10203000964CA540B109840F951FA61FB71F802697
:102040009126A226B326880E991EAA1EBB1ED50174
:10205000C40144E0880F991FAA1FBB1F4A95D1F7FE
:102060005CE1B694A794979487945A95D1F7882AFF
:10207000992AAA2ABB2A800E911EA21EB31E4DA524
:102080005EA56FA578A94F5759406E4878474C0D0B
:102090005D1D6E1D7F1D73016201C026D126E226E3
:1020A000F326C824D924EA24FB24C40ED51EE61E38
:1020B000F71EB701A601EBE0440F551F661F771FFF
:1020C000EA95D1F7F5E1F694E794D794C794FA9599
:1020D000D1F7C42AD52AE62AF72AC80CD91CEA1C4B
:1020E000FB1C49AD5AAD6BAD7CAD4E5D5E496246A1
:1020F0007249440E551E661E771EB901A801482577
:1021000059256A257B254C255D256E257F25440EA6
:10211000551E661E771ED20123013D014C0C5D1C2D
:102120006E1C7F1C29964CAD5DAD6EAD7FAD2997C1
:10213000445F574C6A417240400F511F621F731F2A
:10214000950184010C251D252E253F2504251525E7
:1021500026253725040F151F261F371FB901A80193
:10216000A9E07695679557954795AA95D1F7B7E178
:10217000000F111F221F331FBA95D1F7042B152B07
:10218000262B372B040D151D261D371D49895A890D
:102190006B897C894C5B554161447B45480D591DD9
:1021A0006A1D7B1D4601570184249524A624B7246B
:1021B00080269126A226B326840E951EA61EB71E43
:1021C000B501A40184E0440F551F661F771F8A954F
:1021D000D1F79CE1B694A794979487949A95D1F7F8
:1021E000842A952AA62AB72A800E911EA21EB31E03
:1021F0004D8D5E8D6F8D78A1475550436142744B74
:10220000C40ED51EE61EF71EB301A20140275127BA
:1022100062277327482559256A257B254C0D5D1DAE
:102220006E1D7F1DDB01CA01EBE0880F991FAA1FFD
:10223000BB1FEA95D1F7F5E17695679557954795D8
:10224000FA95D1F7482B592B6A2B7B2B480D591D3A
:102250006A1D7B1DC9A4DAA4EBA4FCA4B0EACB1AC6
:10226000B4EBDB0AB4E4EB0AB9E0FB0A4C0C5D1CEE
:102270006E1C7F1C68017901C824D924EA24FB2440
:10228000C426D526E626F7264C0C5D1C6E1C7F1C4A
:10229000F20123013F01440E551E661E771ECDA894
:1022A000DEA8EFA8F8ACF0E9CF1AF3E4DF0AF0E417
:1022B000EF0AF1E4FF0AC00ED11EE21EF31E9501E3
:1022C00084010427152726273727042515252625C9
:1022D00037250C0D1D1D2E1D3F1D68017901A9E03C
:1022E000F694E794D794C794AA95D1F7B7E1000F75
:1022F000111F221F331FBA95D1F70C291D292E2932
:102300003F29040D151D261D371D2596CCACDDACCF
:10231000EEACFFAC25978AE3C81A81E8D80A84E6B8
:10232000E80A87EDF80AC80CD91CEA1CFB1C4A0114
:102330005B0184249524A624B72480269126A22616
:10234000B3268C0C9D1CAE1CBF1C7501640184E07F
:10235000CC0CDD1CEE1CFF1C8A95D1F79CE1B694D9
:10236000A794979487949A95D1F78C289D28AE28A6
:10237000BF28800E911EA21EB31ECD84DE84EF8482
:10238000F88896E0C91A98EDD90A9EE5E90A95E120
:10239000F90AC40ED51EE61EF71EB301A20140279E
:1023A000512762277327482559256A257B254C0D1F
:1023B0005D1D6E1D7F1D6A017B01EBE0CC0CDD1CF9
:1023C000EE1CFF1CEA95D1F7F5E1769567955795D8
:1023D0004795FA95D1F74C295D296E297F29480D3B
:1023E000591D6A1D7B1DC98CDA8CEB8CFC8CABE70C
:1023F000CA1AAFECDA0AA0E1EA0AABE2FA0A4C0C1C
:102400005D1C6E1C7F1C68017901C824D924EA2454
:10241000FB24C426D526E626F7264C0C5D1C6E1C34
:102420007F1CF20123013F01440E551E661E771EDC
:10243000CDA0DEA0EFA0F8A4FBEFCF1AF2EEDF0AEA
:10244000F7E7EF0AFBEFFF0AC00ED11EE21EF31EF4
:1024500095018401042715272627372704251525EC
:10246000262537250C0D1D1D2E1D3F1D68017901E8
:10247000A9E0F694E794D794C794AA95D1F7B7E169
:10248000000F111F221F331FBA95D1F70C291D29E8
:102490002E293F29040D151D261D371DC9A8DAA8B0
:1024A000EBA8FCA887ECC81A8FE2D80A8BE2E80AEE
:1024B00086E2F80AC80CD91CEA1CFB1C4A015B0125
:1024C00084249524A624B72480269126A226B32608
:1024D0008C0C9D1CAE1CBF1C7501640184E0CC0CEF
:1024E000DD1CEE1CFF1C8A95D1F79CE1B694A794E5
:1024F000979487949A95D1F78C289D28AE28BF2869
:10250000800E911EA21EB31E2196CCACDDACEEACAB
:10251000FFAC21979BE1C91A96E6D90A94E2E90A31
:1025200099E1F90AC40ED51EE61EF71EB301A201F9
:102530004027512762277327482559256A257B257F
:102540004C0D5D1D6E1D7F1D6A017B01EBE0CC0C07
:10255000DD1CEE1CFF1CEA95D1F7F5E17695679539
:1025600057954795FA95D1F74C295D296E297F2912
:10257000480D591D6A1D7B1D2D96CCACDDACEEAC13
:10258000FFAC2D97A8E0CA1AA3E8DA0AADE5EA0A7B
:10259000A0EEFA0A4C0C5D1C6E1C7F1C68017901D0
:1025A000C824D924EA24FB24C426D526E626F72607
:1025B0004C0C5D1C6E1C7F1CF20123013F01440E7C
:1025C000551E661E771ECD88DE88EF88F88CFBE9E5
:1025D000CF1AF9EADF0AF3E5EF0AFBE3FF0AC00EC0
:1025E000D11EE21EF31E950184010427152726271C
:1025F000372704251525262537250C0D1D1D2E1DD5
:102600003F1D68017901A9E0F694E794D794C79437
:10261000AA95D1F7B7E1000F111F221F331FBA95FA
:10262000D1F70C291D292E293F29040D151D261D22
:10263000371DCD84DE84EF84F8888CEBC81A8DEDCD
:10264000D80A86EDE80A8BE0F80AC80CD91CEA1C07
:10265000FB1C4A015B0180949094A094B094802A62
:10266000912AA22AB32A84249524A624B7248C0C68
:102670009D1CAE1CBF1C7501640186E0CC0CDD1CEA
:10268000EE1CFF1C8A95D1F79AE1B694A794979413
:1026900087949A95D1F78C289D28AE28BF28800E64
:1026A000911EA21EB31EC9A4DAA4EBA4FCA499E651
:1026B000C91AD10895EDE90A9CEBF90AC40ED51E9A
:1026C000E61EF71EB301A2014095509560957095E6
:1026D000482959296A297B294027512762277327CE
:1026E0004C0D5D1D6E1D7F1D6A017B01EAE0CC0C67
:1026F000DD1CEE1CFF1CEA95D1F7F6E17695679597
:1027000057954795FA95D1F74C295D296E297F2970
:10271000480D591D6A1D7B1D2996CCACDDACEEAC75
:10272000FFAC2997A9E5CA1AACEDDA0AABE6EA0ACA
:10273000A4E5FA0AC40CD51CE61CF71C28013901D3
:102740004094509460947094442A552A662A772ABB
:10275000482459246A247B244C0C5D1C6E1C7F1C6D
:1027600073016201AFE0CC0CDD1CEE1CFF1CAA95CE
:10277000D1F7B1E17694679457944794BA95D1F71D
:102780004C285D286E287F28440E551E661E771E35
:10279000C9A0DAA0EBA0FCA0B7ECCB1ABFE5DB0A1E
:1027A000BCE6EB0AB3E0FB0AC00ED11EE21EF31E2C
:1027B00095018401009510952095309504291529DF
:1027C0002629372904271527262737270C0D1D1DF5
:1027D0002E1D3F1D680179018BE0F694E794D79494
:1027E000C7948A95D1F795E1000F111F221F331F5F
:1027F0009A95D1F70C291D292E293F29040D151D65
:10280000261D371D2196CCACDDACEEACFFAC21977C
:10281000EDE3CE1AE6EADE0AE4EAEE0AEAE9FE0AA7
:10282000C80CD91CEA1CFB1C4A015B0180949094E3
:10283000A094B094802A912AA22AB32A84249524B1
:10284000A624B7248C0C9D1CAE1CBF1C7501640112
:10285000E6E0CC0CDD1CEE1CFF1CEA95D1F7FAE19A
:10286000B694A79497948794FA95D1F78C289D28CD
:10287000AE28BF28800E911EA21EB31EC98CDA8C12
:10288000EB8CFC8CFEE6CF1AF3E3DF0AF3EFEF0AE2
:10289000F0E7FF0AC40ED51EE61EF71EB301A20123
:1028A0004095509560957095482959296A297B294A
:1028B00040275127622773274C0D5D1D6E1D7F1D1C
:1028C0006A017B01AAE0CC0CDD1CEE1CFF1CAA9562
:1028D000D1F7B6E17695679557954795BA95D1F7B3
:1028E0004C295D296E297F29480D591D6A1D7B1DC4
:1028F000CDA8DEA8EFA8F8AC83E8C81A8BE0D80A08
:1029000080E1E80AF108C40CD51CE61CF71C28017C
:1029100039014094509460947094442A552A662A50
:10292000772A482459246A247B244C0C5D1C6E1C95
:102930007F1C730162018FE0CC0CDD1CEE1CFF1CC0
:102940008A95D1F791E176946794579447949A9534
:10295000D1F74C285D286E287F28440E551E661E30
:10296000771EC988DA88EB88FC889FE2C91A92EA48
:10297000D90A9BE7E90A9AE7F90AC00ED11EE21EBE
:10298000F31E95018401009510952095309504293A
:1029900015292629372904271527262737270C0D1F
:1029A0001D1D2E1D3F1D68017901EBE0F694E79493
:1029B000D794C794EA95D1F7F5E1000F111F221FB4
:1029C000331FFA95D1F70C291D292E293F29040D13
:1029D000151D261D371DCDA4DEA4EFA4F8A8A1EB7C
:1029E000CA1AA1E8DA0AA7E5EA0AA0E9FA0AC80CB5
:1029F000D91CEA1CFB1C4A015B0180949094A094B2
:102A0000B094802A912AA22AB32A84249524A62449
:102A1000B7248C0C9D1CAE1CBF1C75016401A6E084
:102A2000CC0CDD1CEE1CFF1CAA95D1F7BAE1B694C4
:102A3000A79497948794BA95D1F78C289D28AE28AF
:102A4000BF28800E911EA21EB31E2D968CAD9DAD8B
:102A5000AEADBFAD2D9780529941A34DB140840FCB
:102A6000951FA61FB71FB301A20140955095609511
:102A70007095482959296A297B29402751276227BF
:102A80007327840F951FA61FB71F6C017D014AE0B5
:102A9000CC0CDD1CEE1CFF1C4A95D1F7AC01BD012E
:102AA000E6E17695679557954795EA95D1F74C29D4
:102AB0005D296E297F29480D591D6A1D7B1D8DA139
:102AC0009EA1AFA1B8A58C5E9C4BAE4FBC45840DBA
:102AD000951DA61DB71D280139014094509460949E
:102AE0007094442A552A662A772A482459246A244D
:102AF0007B24840D951DA61DB71D6C017D01FFE093
:102B0000CC0CDD1CEE1CFF1CFA95D1F72C013D010D
:102B1000A1E17694679457944794AA95D1F74C28ED
:102B20005D286E287F28440E551E661E771E25964A
:102B30008CAD9DADAEADBFAD25978F559E4EA74FC9
:102B4000B14B800F911FA21FB31F95018401009507
:102B50001095209530950429152926293729042711
:102B6000152726273727800F911FA21FB31F6C013F
:102B70007D011BE0F694E794D794C7941A95D1F79A
:102B80008C019D0185E1000F111F221F331F8A95C3
:102B9000D1F70C291D292E293F29040D151D261DAD
:102BA000371D8D8D9E8DAF8DB8A18E579148AC4A43
:102BB000B840880D991DAA1DBB1D4A015B01809478
:102BC0009094A094B094802A912AA22AB32A8424B3
:102BD0009524A624B724880D991DAA1DBB1D6C0140
:102BE0007D01E6E0CC0CDD1CEE1CFF1CEA95D1F764
:102BF0004C015D01FAE1B694A79497948794FA95F5
:102C0000D1F78C289D28AE28BF28800E911EA21EC9
:102C1000B31E89AD9AADABADBCAD8B5C9D40A54CF0
:102C2000B244840F951FA61FB71FB301A2014095A0
:102C3000509560957095482959296A297B29402724
:102C4000512762277327840F951FA61FB71F6C019A
:102C50007D014AE0CC0CDD1CEE1CFF1C4A95D1F72F
:102C6000AC01BD01E6E17695679557954795EA95E4
:102C7000D1F74C295D296E297F29480D591D6A1D00
:102C80007B1D8D899E89AF89B88D85549D42A84250
:102C9000B54D840D951DA61DB71D28013901409421
:102CA000509460947094442A552A662A772A4824BE
:102CB00059246A247B24840D951DA61DB71D6C0123
:102CC0007D01FFE0CC0CDD1CEE1CFF1CFA95D1F75A
:102CD0002C013D01A1E17694679457944794AA95FD
:102CE000D1F74C285D286E287F28440E551E661E9D
:102CF000771E89A99AA9ABA9BCA98F569C42A9475E
:102D0000B441800F911FA21FB31F9501840100954C
:102D1000109520953095042915292629372904274F
:102D2000152726273727800F911FA21FB31F6C017D
:102D30007D011BE0F694E794D794C7941A95D1F7D8
:102D40008C019D0185E1000F111F221F331F8A9501
:102D5000D1F70C291D292E293F29040D151D261DEB
:102D6000371D61968CAD9DADAEADBFAD6197880D41
:102D7000991DAA1DBB1D61968CAF9DAFAEAFBFAFB5
:102D8000619789819A81AB81BC81800F911FA21FBD
:102D9000B31F89839A83AB83BC830D811E812F81EE
:102DA0003885040D151D261D371D0D831E832F83A9
:102DB000388789859A85AB85BC85840F951FA61FAA
:102DC000B71F89879A87AB87BC87E796AEADBFAD43
:102DD000E797A05CBF4FE796BFAFAEAFE797B0E411
:102DE0002B1A310811F00C94710761960CAD1DADD2
:102DF0002EAD3FAD6197E996AEADBFADE9971896A0
:102E00000D931D932D933C931B9709811A812B8160
:102E10003C811C960D931D932D933C931F970D8120
:102E20001E812F81388550960D931D932D933C93D1
:102E3000539709851A852B853C8554960D931D93D0
:102E40002D933C935797E7968EAD9FADE797C85863
:102E5000DF4F0FB6F894DEBF0FBECDBFDF91CF912D
:102E60001F910F91FF90EF90DF90CF90BF90AF90A8
:102E70009F908F907F906F905F904F903F902F909A
:102E800008950F931F93CF93DF93EC01062F142F18
:102E900060E08E850E9493013C852D858091AD0276
:102EA000882381F09FB7F8948091AD02813081F53D
:102EB0008DB38093A8024DB38091AC02809584239A
:102EC0008DBB9FBF3CBD2DBD0EBD00000DB407FEE8
:102ED000FDCF8EB51EBD00000DB407FEFDCF1EB5A3
:102EE0008091AD02882351F09FB7F8942091AD02F4
:102EF0008091A802213079F48DBB9FBF61E08E855F
:102F00000E949301812FDF91CF911F910F9108951E
:102F10009093A802D7CF8FBFF1CFCF93DF93EC016F
:102F2000429714F0C1E1D0E044E86DEC8FEF9EE1F0
:102F30000E944117C230D10514F4C2E0D0E0C25063
:102F40004C2F406869E88FEF9EE1DF91CF910C94A0
:102F50004117CF93DF93672BB1F4EC010F9714F077
:102F6000CEE0D0E044E86DEC8FEF9EE10E94411787
:102F7000D7FDC0E04C2F406769E88FEF9EE1DF91FD
:102F8000CF910C944117DF91CF910C948D17AF9294
:102F9000BF92CF92DF92EF92FF920F931F93CF9346
:102FA0006093131F7093141F8093151F9093161F27
:102FB0006B017C01FF0CCC08DC2C76019B01AC0181
:102FC0006C2D7C2D8C2D9C2D03E10E94A52DA12C18
:102FD000E8E4BE2EF8EECF2EDD24D394E12CF12CC4
:102FE00000E010E00E94482DC22FC22ED32E7A019D
:102FF000A7016627772766E88FEF9EE10E944117B9
:1030000077276F2D5E2D4D2D67E88FEF9EE10E9493
:1030100041174C2F68E88FEF9EE1CF911F910F91E0
:10302000FF90EF90DF90CF90BF90AF900C9441173E
:1030300040E861E88FEF9EE10E9441179FB7F89446
:103040008091AE02882319F081508093AE02809166
:10305000AE02811105C08CB58F7B8CBD1092AD0284
:103060009FBF1092571E089540E00C944117CF92D5
:10307000DF92EF92FF920F931F93CF93DF936AE15A
:103080008FEF9EE10E943418C82FD0E069E18FEFE6
:103090009EE10E943418682F880F770B880B990BDC
:1030A0000E942C2B20E030E040E85EE30E948B2B56
:1030B0000E94C22C6B018B016091131F7091141F31
:1030C0008091151F9091161F0E942C2B24ED30E843
:1030D00043E45EE40E94252BBE0187FD10C06D59BC
:1030E000710917FF0FC06C0D7D1DCB01DF91CF91D2
:1030F0001F910F91FF90EF90DF90CF900895645A49
:103100007109EFCF072E000C880B990B0E942C2B16
:1031100020EB32E748E85FE30E948B2B0E94C22C31
:10312000E4CF43E861E88FEF9EE10E94411762E13E
:103130008FEF9EE10E94341883FFF9CF48E062E9E7
:103140008FEF9EE10E94411781E090E00895CF92B9
:10315000DF92EF92FF926EE18FEF9EE10E943418B2
:1031600082958F70CC24C394D12C02C0CC0CDD1C72
:103170008A95E2F70D2C000CEE08FF086DE18FEF49
:103180009EE10E94341890E044E0959587954A9519
:10319000E1F78A30910534F5FC01EE0FFF1FE80FCF
:1031A000F91FEC5DFD4F608171818281082E000C5A
:1031B000990B28EE33E040E050E00E945F2CC701FD
:1031C000B6010E945F2C213131054105510574F093
:1031D0004CE066EA8FEF9EE1FF90EF90DF90CF909A
:1031E0000C94411760E070E0CB01E3CF44E0F1CFF5
:1031F000CF93DF93EC01863091052CF08D30910553
:1032000034F5069731F545EC61EB8FEF9EE10E94B6
:1032100041174CE067EB8FEF9EE10E944117C6E03B
:10322000D0E06EE18FEF9EE10E9434188F7094E041
:10323000CC0FDD1F9A95E1F74C2F482B6EE98FEFED
:103240009EE10E944117DF91CF910C94A718CCE02A
:10325000D0E043EC61EB8FEF9EE10E9441174AE022
:1032600067EB8FEF9EE10E944117DBCFCF93DF9397
:10327000EC01099714F0C8E0D0E06DE18FEF9EE11A
:103280000E943418C530D10514F4C5E0D0E024976D
:10329000CC0FDD1F482F417F4C2B6DE98FEF9EE156
:1032A000DF91CF910C94411710921A1F1092191FA1
:1032B0006DE18FEF9EE10E943418482F4E7F6DE93B
:1032C0008FEF9EE10C94411781E090E090931A1FDC
:1032D0008093191F6DE18FEF9EE10E943418482FF3
:1032E00041606DE98FEF9EE10C944117CF93DF931E
:1032F000EC0141E861E88FEF9EE10E944117CD2B80
:1033000099F00E94641940E06DE88FEF9EE10E9401
:10331000411740E062EA8FEF9EE10E94411781E091
:1033200090E0DF91CF9108950E945419ECCF0F9354
:103330001F93CF93DF9366E08FEF9EE10E943418D6
:10334000D82F67E08FEF9EE10E943418C82F68E005
:103350008FEF9EE10E9434184C2F50E070E060E047
:10336000762F652F542F44276D2B8A019B01082B44
:10337000C901B80120E038E448EE51E00E941B2D5D
:1033800003E10E94C02D2093270A3093280A40931E
:10339000290A50932A0ADF91CF911F910F91089526
:1033A000CF92DF92EF92FF92CF93DF936091230A47
:1033B0007091240A8091250A9091260A0E942C2B54
:1033C0006B017C0120E030EC43EF55E40E94252B9B
:1033D000D0E0C0E018160CF065C020E030E842E212
:1033E00056E4C701B6010E94252BC1E0D0E01816B3
:1033F0000CF058C020E030EC43E756E4C701B601BA
:103400000E94252BC2E0D0E018160CF04BC020E043
:1034100030E842EA56E4C701B6010E94252BC3E01A
:10342000D0E018160CF03EC020E034E244EF56E441
:10343000C701B6010E94252BC4E0D0E0181694F510
:1034400020E034EE42E257E4C701B6010E94252B8A
:10345000C5E0D0E0181634F520E034E244E757E444
:10346000C701B6010E94252BC6E0D0E01816D4F49F
:1034700020E034E244EF57E4C701B6010E94252B57
:10348000C7E0D0E0181674F420E034E244E758E4D2
:10349000C701B6010E94252BC9E0D0E0181614F030
:1034A000C8E0D0E06DE18FEF9EE10E9434188F708C
:1034B00044E0CC0FDD1F4A95E1F74C2F482B6DE916
:1034C0008FEF9EE10E9441170E94A7188091571E1E
:1034D000882319F16DE18FEF9EE10E94341890E08E
:1034E00034E0959587953A95E1F78A309105E4F4B3
:1034F000FC01EE0FFF1FE80FF91FEC5DFD4F80810F
:103500009181A2810A2E000CBB0B8093230A909319
:10351000240AA093250AB093260ADF91CF91FF9049
:10352000EF90DF90CF90089580E090E0DC01EDCF48
:1035300068E18FEF9EE10E9434189FB7F8944091A4
:10354000591E50915A1E60915B1E70915C1E9FBF68
:10355000409318085093190860931A0870931B0839
:1035600080FF2AC081E08093B3028093B2028093EF
:10357000B1028091AF029091B0022091B30221116B
:1035800008C02091B202211104C02091B10222236F
:1035900001F18F309105B8F401969093B0028093B9
:1035A000AF0281E08093541E8091531E8823F1F076
:1035B00061E08CE00C9493011092B3021092B2027D
:1035C0001092B102D6CF81E08093541E8093531E97
:1035D000EBCF009741F001979093B0028093AF0238
:1035E0001092541EE1CF1092531EFACF0C941C0679
:1035F000CF93DF9362E18FEF9EE10E943418C82FD2
:10360000482F62E98FEF9EE10E944117C5FD2DC052
:103610001092181F1092171F8091191F90911A1F56
:1036200062E2892B09F463E18FEF9EE10E94341876
:10363000C82FD0E060E18FEF9EE10E943418482F40
:103640006DE88FEF9EE10E944117E0911B1FF09102
:103650001C1F309711F0CE01199540E06DE88FEFF7
:103660009EE1DF91CF910C944117DF91CF910895A6
:1036700008950F931F93CF93DF93EC01E881F981B5
:103680000084F185E02D1995892BB1F06DE0CE0114
:103690000E943418082F60E0CE010E943418182FC1
:1036A000402F6DE8CE010E944117812F90E0DF91FD
:1036B000CF911F910F9108958FEF9FEFF8CFCF9388
:1036C000DF93EC01E881F9810084F185E02D199503
:1036D000892B69F0888D998D0196998F888F60E08C
:1036E000CE010E94341890E0DF91CF9108958FEFC2
:1036F0009FEFFACFCF93DF93EC012097E1F0219772
:103700008091AA029091AB028C3F9140A0F48FEF80
:103710009EE10E945F1B2091AA023091AB02A90199
:103720004F5F5F4F5093AB024093AA02255E3C4F20
:10373000F9018083E2CFDF91CF9108950F931F931A
:10374000CF93DF93EC018091200A811178C08FEF35
:103750009EE10E945F1B21974091000280FF55C0AF
:103760009C0154E0359527955A95E1F72F70332742
:103770004F3FD1F41092AB021092AA0220930002A4
:103780000E943718909302028093010269E18FEF43
:103790009EE10E9434188093A902CE01DF91CF915F
:1037A0001F910F910C947A1B2413E4CF0E943718B9
:1037B0002091010230910202820F931F97FD019622
:1037C0009595879590930202809301020091A9023A
:1037D00010E069E18FEF9EE10E943418800F912F75
:1037E000911D959587958093A902CE010E947A1B21
:1037F0008FEF809300020E94E3050E94D305DF91C2
:10380000CF911F910F910C94E4044F3F39F0109227
:10381000AB021092AA028FEF809300020E94371829
:10382000909302028093010269E18FEF9EE10E9472
:1038300034188093A902CE010E947A1BDCCF10922B
:10384000AB021092AA02EACFCF93DF93EC0163E1BF
:103850000E94341890E0288D398D821B930BDF91E4
:10386000CF910895AF92BF92CF92DF92FF920F93C4
:103870001F93CF93DF936C015B01EA0162E20E9428
:103880003418F82E90E09C012C0F3D1F2F3F31057E
:1038900029F020F0CFEFD0E0C81BD90B8501AC0E8A
:1038A000BD1E0A151B0541F0F80141918F0160E82A
:1038B000C6010E944117F5CF4C2F4F0D62EAC60199
:1038C0000E944117CE01DF91CF911F910F91FF9080
:1038D000DF90CF90BF90AF900895CF93DF931F926A
:1038E000CDB7DEB76983DC01ED91FC910280F381F5
:1038F000E02D41E050E0BE016F5F7F4F19950F90C2
:10390000DF91CF91089590E080E008958091B50215
:10391000823A49F470E060E08091160290911702BB
:103920000E94A9170895833AA9F3843A99F3873A34
:1039300039F480911602909117020E948D17089514
:10394000883AB9F3893AA9F3833B99F3843B89F325
:10395000883B79F3893B69F3843C59F3893C31F422
:1039600080911602909117020C948D17843EC1F33A
:10397000893EB1F38E3FA1F38F3F41F470E060E0E8
:1039800080911602909117020C94A9170895CF9375
:1039900080911E0A811103C00E9454190CC0C0916D
:1039A0001F0ACC23C9F30E9464194C2F62EA8FEFDF
:1039B0009EE10E94411745E861E88FEF9EE1CF91BB
:1039C0000C944117CF92DF92EF92FF92CF93DF9347
:1039D0000E94B804D091571ED11190C1809113025A
:1039E000811185C1C091521ECC2309F480C1C090C1
:1039F000270AD090280AE090290AF0902A0A61E06C
:103A000080910D1F0E941F0261E080910D1F0E9496
:103A1000930180910F1F9091101F8F3F9807C9F05D
:103A200061E00E941F0260E080910F1F0E949301DD
:103A30006AE070E080E090E00E944C0361E08091D9
:103A40000F1F0E9493016AE070E080E090E00E9406
:103A50004C03DFB7F8948091AE02811127C0EDE1ED
:103A6000F2E08491E3E6F2E09491E82FF0E0EE0FCB
:103A7000FF1FEC54FE4FA591B491EC91E92321F482
:103A800061E085E30E94930161E085E30E941F02EB
:103A90008CB580618CBD8CB580648CBD61E084E3A5
:103AA0000E941F0261E083E30E941F028091AE0228
:103AB0008F5F8093AE02DFBF62E48FEF9EE10E94D2
:103AC0003418823181F081E00E94610590E080E04D
:103AD0000E945E06D0E08D2FDF91CF91FF90EF9096
:103AE000DF90CF90089540E861E88FEF9EE10E945B
:103AF0004117C701B6010E94C71740E06EE88FEF7B
:103B00009EE10E94411740E06FE88FEF9EE10E9426
:103B100041176CE08FEF9EE10E943418482F4360FC
:103B20006CE88FEF9EE10E94411744E066EA8FEF58
:103B30009EE10E94411782E090E00E948D1741E8CB
:103B400061E88FEF9EE10E94411781E08093571E4C
:103B50000E94861C0E94D0198091210A9091220A0D
:103B60000E94F81880911402909115020E94361953
:103B70000E9497196EE18FEF9EE10E943418482F42
:103B800044606EE98FEF9EE10E9441178EE99BE150
:103B900090931C1F80931B1F60E08091111F0E9457
:103BA0001F0240E060EC8FEF9EE10E9441172091E0
:103BB000111F3091121F80E02230310551F081E059
:103BC0002330310531F0C9014297049790F487E121
:103BD000821B2FB7F894823009F43FC060F4882329
:103BE00009F441C0813071F082E08093AD0280E041
:103BF0000AC08FEFEECF8430A1F188F18530A1F7B4
:103C000088E001C080E29091AC02892B8093AC02E5
:103C10008091AD02811103C081E08093AD022FBF7E
:103C20002091111F3091121F22303105F1F488EFDD
:103C30009AE1909304028093030280916A0083606A
:103C400080936A00EC9A0E94C71C0E94500583E092
:103C500090E00E942006DC2F3ECF81E0D4CF82E0AE
:103C6000D2CF84E0D0CF80E1CECF2330310569F4CC
:103C700088EF9AE1909306028093050280916A0092
:103C80008C6080936A00ED9ADECFC9014297049759
:103C9000D0F687E1821BE82FF0E0EE0FFF1FED5F0B
:103CA000FD4F28EF3AE131832083843091F0853055
:103CB000B9F0833039F080916900836080936900A6
:103CC000E89AC1CF809169008C6080936900E99A7D
:103CD000BACF80916900806380936900EA9AB3CF7C
:103CE00080916900806C80936900EB9AACCF0E9450
:103CF000500583E090E00E94FF05EDCE0E94500544
:103D0000EACE0C94492C1F920F920FB60F921124F9
:103D10002F933F938F939F93AF93BF938091591E9F
:103D200090915A1EA0915B1EB0915C1E3091581E5E
:103D300023E0230F2D3758F50196A11DB11D2093C7
:103D4000581E8093591E90935A1EA0935B1EB093E9
:103D50005C1E80915D1E90915E1EA0915F1EB091D1
:103D6000601E0196A11DB11D80935D1E90935E1E85
:103D7000A0935F1EB093601EBF91AF919F918F91F2
:103D80003F912F910F900FBE0F901F90189526E82E
:103D9000230F0296A11DB11DD2CF1F920F920FB615
:103DA0000F9211240BB60F922F933F934F935F9373
:103DB0006F937F938F939F93AF93BF93EF93FF93F3
:103DC000E0911102F09112021995FF91EF91BF91CC
:103DD000AF919F918F917F916F915F914F913F91A3
:103DE0002F910F900BBE0F900FBE0F901F90189544
:103DF0001F920F920FB60F9211240BB60F922F93B2
:103E00003F934F935F936F937F938F939F93AF9362
:103E1000BF93EF93FF93E0910F02F0911002199579
:103E2000FF91EF91BF91AF919F918F917F916F9192
:103E30005F914F913F912F910F900BBE0F900FBE4E
:103E40000F901F9018951F920F920FB60F9211248A
:103E50000BB60F922F933F934F935F936F937F9384
:103E60008F939F93AF93BF93EF93FF93E0910502DE
:103E7000F09106021995FF91EF91BF91AF919F913B
:103E80008F917F916F915F914F913F912F910F9003
:103E90000BBE0F900FBE0F901F9018951F920F92A0
:103EA0000FB60F9211240BB60F922F933F934F939F
:103EB0005F936F937F938F939F93AF93BF93EF9392
:103EC000FF93E0910302F09104021995FF91EF91A5
:103ED000BF91AF919F918F917F916F915F914F9122
:103EE0003F912F910F900BBE0F900FBE0F901F9020
:103EF00018951F920F920FB60F9211240BB60F92C6
:103F00002F933F934F935F936F937F938F939F93E1
:103F1000AF93BF93EF93FF93E0910D02F0910E02E8
:103F20001995FF91EF91BF91AF919F918F917F91E3
:103F30006F915F914F913F912F910F900BBE0F901A
:103F40000FBE0F901F9018951F920F920FB60F92F1
:103F500011240BB60F922F933F934F935F936F9360
:103F60007F938F939F93AF93BF93EF93FF93E091D2
:103F70000B02F0910C021995FF91EF91BF91AF9157
:103F80009F918F917F916F915F914F913F912F9171
:103F90000F900BBE0F900FBE0F901F9018951F92A1
:103FA0000F920FB60F9211240BB60F922F933F93DF
:103FB0004F935F936F937F938F939F93AF93BF9331
:103FC000EF93FF93E0910902F0910A021995FF9196
:103FD000EF91BF91AF919F918F917F916F915F9181
:103FE0004F913F912F910F900BBE0F900FBE0F90EE
:103FF0001F9018951F920F920FB60F9211240BB6B7
:104000000F922F933F934F935F936F937F938F9371
:104010009F93AF93BF93EF93FF93E0910702F091CB
:1040200008021995FF91EF91BF91AF919F918F91E8
:104030007F916F915F914F913F912F910F900BBEA8
:104040000F900FBE0F901F9018951F920F920FB6F2
:104050000F9211240BB60F922F933F934F935F93C0
:104060006F937F938F939F93AF93BF93EF93FF9340
:1040700081E69EE10E94F303FF91EF91BF91AF9122
:104080009F918F917F916F915F914F913F912F9170
:104090000F900BBE0F900FBE0F901F9018951F92A0
:1040A0000F920FB60F9211240BB60F922F938F938E
:1040B0009F93EF93FF93E091711EF091721E8081A8
:1040C000E091771EF091781E82FD1DC09081809155
:1040D0007A1E8F5F8F7320917B1E821741F0E091D3
:1040E0007A1EF0E0EF59F14E958F80937A1EFF9182
:1040F000EF919F918F912F910F900BBE0F900FBE5C
:104100000F901F9018958081F2CF1F920F920FB6DB
:104110000F9211240BB60F922F933F934F935F93FF
:104120006F937F938F939F93AF93BF93CF93EF93AF
:10413000FF938091B402811127C081E08093B40283
:10414000C4E181E69EE10E94DD03892BD9F08FB79F
:10415000F89440914E1E50914F1E20914A1E30916E
:104160004B1E4217530721F54091501E5091511E8E
:1041700020914C1E30914D1E42175307C9F48FBF3A
:10418000C150F9F61092B402FF91EF91CF91BF9117
:10419000AF919F918F917F916F915F914F913F91DF
:1041A0002F910F900BBE0F900FBE0F901F90189580
:1041B0004091501E5091511E20914E1E30914F1E25
:1041C0002150310942175307D1F28FBF81E69EE19A
:1041D0000E94BB032FB7F894E091501EF091511E3E
:1041E00080834091501E5091511E80914C1E9091A1
:1041F0004D1E4817590751F480914A1E90914B1E4D
:104200009093511E8093501E2FBFBACF8091501EA5
:104210009091511E0196F4CF88E198E00FB6F89482
:10422000A895809360000FBE909360000E94FB05EC
:104230000E941C06FBCF1F93CF93DF93EC01162F38
:104240000E94492C181739F0612FCE01DF91CF91D0
:104250001F910C94512CDF91CF911F910895E1E6AD
:10426000FEE11382128288EE93E0A0E0B0E0848346
:104270009583A683B78386E492E09183808385EC5F
:1042800090E09587848784EC90E09787868780EC20
:1042900090E0918B808B81EC90E0938B828B82EC11
:1042A00090E0958B848B86EC90E0978B868B118EBB
:1042B000128E138E148E81E08093FE1EEFEFFEE1CE
:1042C0001382128228E532E03183208390E59487BF
:1042D00085878AE090E09787868789E090E0918BD8
:1042E000808B82E090E0938B828B148A158A168AE9
:1042F000178A118E108E138E128E158E148E1482C4
:104300001582168217820895CF93DF93CDB7DEB75B
:10431000C859D1090FB6F894DEBF0FBECDBF78944F
:1043200084B5826084BD84B5816084BD85B58260BA
:1043300085BD85B5816085BD80916E00816080936B
:104340006E001092810080918100826080938100D4
:1043500080918100816080938100809180008160E4
:10436000809380008091B10084608093B10080913F
:10437000B00081608093B000809191008260809352
:1043800091008091910081608093910080919000D4
:104390008160809390008091A10082608093A10051
:1043A0008091A10081608093A1008091A000816034
:1043B0008093A000809121018260809321018091EF
:1043C000210181608093210180912001816080938F
:1043D000200180917A00846080937A0080917A0035
:1043E000826080937A0080917A00816080937A0065
:1043F00080917A00806880937A001092C100809149
:104400007B00877F80937B0080E480937C00809199
:104410007A00806480937A0080917A0086FDFCCFD8
:104420006091780070917900072E000C880B990B31
:10443000611571058105910511F00E941C2BE7E1C2
:10444000F5E081E093E0DF019C011D9221503040B6
:10445000E1F7F0934B1EE0934A1EF093511EE09358
:10446000501EF0934F1EE0934E1E87E198E090930C
:104470004D1E80934C1EE091711EF091721E82E0E1
:104480008083E0916D1EF0916E1E1082E0916F1E90
:10449000F091701E80E180831092791EE091751E6C
:1044A000F091761E86E08083E091731EF091741E79
:1044B000808180618083E091731EF091741E808101
:1044C00088608083E091731EF091741E8081806803
:1044D0008083E091731EF091741E80818F7D8083B4
:1044E0001092900089E18093910080E89EE3909380
:1044F00097008093960080E28093710061E08CE0E9
:104500000E941F0261E08DE00E941F02EBE1F3E0D8
:104510008CEF91E0DF019C011D9221503040E1F7CA
:10452000EBE2FAE084E0DF011D928A95E9F7EFE221
:10453000FAE080E094E1DF019C011D9221503040BF
:10454000E1F7E9EEF2E082E3DF01282F1D922A95E0
:10455000E9F7F093411EE093401EF093471EE0936D
:10456000461EF093451EE093441E29E133E030934C
:10457000431E2093421EE7EBF2E0DF011D928A9575
:10458000E9F7F093331EE093321EF093391EE09367
:10459000381EF093371EE093361E87EE92E090931C
:1045A000351E8093341E85E090E090930E1F80931B
:1045B0000D1F84E090E09093101F80930F1F82E006
:1045C00090E09093121F8093111F8091211F811101
:1045D00001C083E0282F80FF69C182E08093B6028A
:1045E0008091B6028150823008F074C283ED9FE062
:1045F0000E94811E833709F06DC188E39FE00E940D
:10460000811E833009F063C189E39FE00E94811E0F
:104610008093B5028E3F08F45DC18AE39FE00E945B
:10462000811E81508E3F08F055C18BE090E00E94C2
:10463000E42D6C018C01E8E3EE2EEFE0FE2EC701C5
:104640000E94811EF80181938F01FFEFEF1AFF0A8C
:1046500023E4E2162FE0F20691F780E190E00E9459
:10466000E42D8C0181E093E2A5E4B7E689879A877F
:10467000AB87BC8789E89BEAADECBFEE8D879E8750
:10468000AF87B88B8EEF9CEDAAEBB8E9898B9A8B3C
:10469000AB8BBC8B86E794E5A2E3B0E18D8B9E8B60
:1046A000AF8BB88F1D821E821F821886FE01E75ACB
:1046B000FF4F80E4DF011D928A95E9F7CE018F5A02
:1046C0009F4F28E0FC0111922A95E9F72BE0F601B3
:1046D000DE01599601900D922A95E1F720E82CA36E
:1046E000FE01B5962CE2DF011D922A95E9F748E517
:1046F00050E060E070E049835A836B837C8328E557
:10470000FC01208340E450E0BE01675E7F4F80558E
:1047100091090E94910639852A859B858C85D8014F
:104720003C9311962C93119712969C931297139683
:104730008C9313973D852E859F85888914963C938D
:10474000149715962C93159716969C931697179673
:104750008C93179739892A899B898C8918963C9361
:10476000189719962C9319971A969C931A971B963B
:104770008C931B973D892E899F89888D1C963C932D
:104780001C971D962C931D971E969C931E971F9603
:104790008C934801BB24B394C7010E94811EF4018D
:1047A00091914F018913B12CFFEFEF1AFF0A23E516
:1047B000E2162FE0F20681F7C8010E94802EC601A2
:1047C0000E94802EBB2009F487C081E08093521E96
:1047D0008FED9FE00E94811E833709F07DC084ED3C
:1047E0009FE00E94811E90E09093220A8093210A0C
:1047F00085ED9FE00E94811E90E0909315028093CA
:10480000140286ED9FE00E94811E90E090931702B3
:10481000809316028BED9FE00E94811E182F8CED75
:104820009FE00E94811E90E0B0E0A0E07C01DD24CA
:10483000CC24F12A8DED9FE00E94811E182F8EED71
:104840009FE00E94811EC82AD12AC092270AD092D6
:10485000280AE092290AF0922A0A87ED9FE00E9436
:10486000811E182F88ED9FE00E94811E90E0B0E02D
:10487000A0E07C01DD24CC24F12A89ED9FE00E9498
:10488000811E182F8AED9FE00E94811EC82AD12A1E
:10489000C092230AD092240AE092250AF092260AB6
:1048A00082E1809318020E94E21C16C083E022FD80
:1048B00095CE23FF02C081E091CE42E250E066E651
:1048C00072E081E69EE10E947F030E944706803FDE
:1048D00009F49ACE1092521E812C34E1932E412C71
:1048E000512C32015394AA24A39454E1B52E809103
:1048F000571E882309F407C22FB7F8948091591ED8
:1049000090915A1EA0915B1EB0915C1E2FBF4091EA
:1049100018085091190860911A0870911B08841B9F
:10492000950BA60BB70B0397A105B10510F00E94DC
:10493000981A8091561E882309F415C11091551EAE
:10494000111102C00E94981A8091541E8111D7C182
:104950008091531E8111D3C1112331F062E370E0C5
:1049600080E090E00E944C030E94981A8091541EAF
:104970008111F9C01092551E8091180A8111EBC067
:1049800081E08093180A4FB7F8942091441E30912B
:10499000451E8091461E9091471E4FBF281739072C
:1049A00009F4D9C0E091441EF091451E8091421E49
:1049B0009091431EE817F90709F093C08091401EBB
:1049C0009091411E9093451E8093441E2081318119
:1049D000E091361EF091371E8091341E9091351E65
:1049E000E817F90709F084C08091321E9091331EB8
:1049F0009093371E8093361E00811181C801019764
:104A00008C3F914008F0BFCFECE1F8E02C513840EA
:104A1000C9018E0F9F1FB4010E94F82CDC01A15D1B
:104A2000B54F8C918193CF018C519840801791079D
:104A300078F38091571E882309F485C08091200A5D
:104A400081115DC00E94FB050E94CD2AA301920145
:104A50000E945F2C607F362E0F3F110510F0689486
:104A600030F890E080E00E947619632D8FEF9EE190
:104A70000E946D1C9CE1C92E98E0D92EEE24E3948F
:104A8000F12CD6016D916D018FEF9EE10E946D1C9E
:104A9000BFEFEB1AFB0AEFEFEE16F10471F40E9480
:104AA000911890E080E00E947619632D8FEF9EE1CF
:104AB0000E946D1CEE24E394F12CC6018C519840A9
:104AC00080179107F0F20E9491180E94F7050E944A
:104AD000C71C59CF1092521E4EE150E069E872E0B7
:104AE000F0CEE091441EF091451ECF0102966ACFB0
:104AF000E091361EF091371ECF01029679CF0E94C9
:104B0000FB050F3F110519F010F00FEF10E0809139
:104B10001E0A811116C090E080E00E947619BCE167
:104B2000EB2EB8E0FB2ED7016D917D018FEF9EE15A
:104B30000E946D1CC7018C5198408017910798F313
:104B4000C2CFC801EACF82E00E94610585E090E013
:104B50000E945E0618CF1092561E10923F1E1092B1
:104B60003E1E1092180A4FB7F89420914E1E3091B5
:104B70004F1E8091501E9091511E4FBF281739072C
:104B800009F4B0C481E08093491EFF24F394AEEF92
:104B9000EA2E4FB7F89420914E1E30914F1E80910F
:104BA000501E9091511E4FBF2817390709F498C421
:104BB000E0914E1EF0914F1E80914C1E90914D1E23
:104BC000E817F90709F00AC180914A1E90914B1E1F
:104BD00090934F1E80934E1E10818091481E882313
:104BE00009F483C4103C09F01AC1809119028111A3
:104BF0007FC41092481E8091441E9091451E4091A2
:104C0000401E5091411E8417950761F42091461E65
:104C10003091471E8091421E9091431E28173907FC
:104C200009F4B7CF2091461E3091471E8091441E53
:104C30009091451E02972817390709F4AACF809151
:104C40003E1E90913F1E8115944108F0A2CF209105
:104C50003C1E30913D1E80913A1E90913B1E019763
:104C600010F48FEF93E12817390709F4C4C028170F
:104C7000390708F0BAC0821B930B0196009709F41C
:104C800088CF6091561E6F5F6093561EE091461E5E
:104C9000F091471E318320836091461E7091471E1C
:104CA0002091421E3091431E6217730709F0A6C07F
:104CB0005093471E4093461EE091381EF091391ED6
:104CC000918380832091381E3091391E8091341E4B
:104CD0009091351E2817390709F09BC08091321E2C
:104CE0009091331E9093391E8093381E80913A1E06
:104CF00090913B1E90933D1E80933C1E4ACF81E0D5
:104D00008093551E30CF80911A0A90911B0AA09172
:104D10001C0AB0911D0A0196A11DB11D2091521EC1
:104D2000222369F1893FEAE29E07A105B10548F413
:104D300080931A0A90931B0AA0931C0AB0931D0A31
:104D400012CF10921A0A10921B0A10921C0A10928B
:104D50001D0A6091FE1E81E0623018F0683218F082
:104D60008FEF8093190A8091190A680F6093FE1ED5
:104D700070E08CE00E9450020E94F705F4CE893F5B
:104D8000FAE29F07A105B10558F480931A0A90939F
:104D90001B0AA0931C0AB0931D0A0E941818E3CEA8
:104DA00010921A0A10921B0A10921C0A10921D0AE5
:104DB0006091FE1E81E0623018F0683218F08FEFCB
:104DC0008093190A8091190A680F6093FE1E70E0A3
:104DD0008DE00E9450020E941C06DFCFE0914E1E23
:104DE000F0914F1ECF010196F3CEB501621B730BFC
:104DF000860F971F43CF81E090E043CF2091461E5E
:104E00003091471E2E5F3F4F3093471E2093461E22
:104E100053CF8091381E9091391E029663CF209116
:104E2000301E3091311E2C3F81E0380708F0B1CEA2
:104E3000909119022115310529F49E3F19F4109320
:104E40001902A7CE911144C01B3D19F4F0922F1EF8
:104E5000A0CE80912F1E882349F01C3D21F01D3DDE
:104E600019F41BED01C010EC10922F1E8091561EFC
:104E7000883108F08ECE80913E1E90913F1E8115A4
:104E8000944108F086CE80913E1E90913F1E01967F
:104E900090933F1E80933E1E80913A1E90913B1E40
:104EA0009C012F5F3F4F30933B1E20933A1E815D44
:104EB000954FFC01108380913A1E90913B1E811505
:104EC000944109F066CE10923B1E10923A1E61CEBC
:104ED000913009F04AC01B3DD9F490932F1E809168
:104EE000301E9091311E049709F053CE60912B0A29
:104EF00070912C0A80912D0A90912E0A0E94142DF7
:104F00006115710581059105D9F40E94890541CE8D
:104F100080912F1E882349F01C3D21F01D3D19F47E
:104F20001BED01C010EC10922F1EC9010196909349
:104F3000311E8093301E255D354FD9011C93CFCF94
:104F40006093270A7093280A8093290A90932A0A6B
:104F5000209118022131C9F62091571E2223A9F26F
:104F60000E94C7170E949719D0CF923009F048C00D
:104F70001B3DD9F4F0922F1E8091301E9091311E6E
:104F8000049709F006CE60912B0A70912C0A80914B
:104F90002D0A90912E0A0E94142D6115710581052C
:104FA0009105D9F40E94AE05F4CD80912F1E88237F
:104FB00049F01C3D21F01D3D19F41BED01C010EC22
:104FC00010922F1EC90101969093311E8093301EBE
:104FD000255D354FF9011083CFCF6093230A70937D
:104FE000240A8093250A9093260A80911802813121
:104FF000C9F68091571E8823A9F20E94D019D2CFFA
:105000009330C9F41F3F19F40E941A05C2CD123122
:1050100008F011E1812F90E090931702809316021F
:1050200080911802813181F78091571E882361F3A6
:105030000E94861CE9CF9430F9F41F3F19F40E94B6
:105040003E05A7CD86E090E0163038F0812F90E045
:105050008D30910514F08CE090E09093220A8093BB
:10506000210A20911802213151F72091571E222345
:1050700031F30E94F818E3CF9530F9F41F3F19F48B
:105080000E942C0586CD85E090E0153038F0812F08
:1050900090E08930910514F088E090E0909315023B
:1050A0008093140220911802213151F72091571E4C
:1050B000222331F30E943619E3CF9930B9F41093CB
:1050C0001F0A112381F0F0921E0A80EC90E00E94EA
:1050D000620489E090E00E946204612F81E69EE113
:1050E0000E9415042BC010921E0AEFCF963081F457
:1050F0001F3F19F40E9450054CCD111103C00E94AE
:105100001818F8CF113009F044CD0E94E21CF2CFFC
:105110009132C9F480EC90E00E94620481E290E058
:105120000E94620480E00E94750580E00E9475057F
:1051300080E00E94750580E00E94750580EC90E09B
:105140000E94620426CD923239F480EC90E00E94F5
:10515000620482E290E0E4CF933219F40E94E30506
:1051600018CD973081F40E94B80480EC90E00E9442
:10517000620487E090E00E9462048091130290E054
:105180000E946204DBCF903329F4812F90E00E94CB
:105190002006FFCC903491F48091571E10E08823B4
:1051A00031F06CE28FEF9EE10E943418182F80ECF2
:1051B00090E00E94620480E490E08DCF983071F41A
:1051C000133709F0E6CC80EC90E00E94620488E09E
:1051D00090E00E94620486E490E0D2CF9E30C1F459
:1051E000113089F41093200A80EC90E00E94620450
:1051F0008EE090E00E9462048091200A882331F1C1
:1052000081E090E0BDCF1111EFCF1092200AECCFDA
:105210009F30F9F48091561E883180F480913E1EB3
:1052200090913F1E8115944148F480EC90E00E94DB
:1052300062048FE090E00E946204E2CF80EC90E094
:105240000E9462048FE090E00E94620490E080E09F
:1052500097CF9935A9F4183F09F09BCC82E390E0F1
:105260000E945E0608E31FE06FEFC8010E941B2149
:105270000F5F1F4F011520E11207B1F70E940C21AB
:10528000953521F4183F09F084CCF8CF9135B1F46D
:1052900080EC90E00E94620481E590E00E9462044C
:1052A00008E31FE0C8010E94811E0E9475050F5F80
:1052B0001F4F011530E11307A9F740CF9235D9F5FB
:1052C0001B3DE9F4F0922F1E8091301E9091311E0B
:1052D000029709F05ECC00912C0A10912B0A83ED05
:1052E0009FE00E94811E833711F1183C00F5812F49
:1052F00090E0602F885C904F0E941B214ACC8091E7
:105300002F1E882349F01C3D21F01D3D19F41BED93
:1053100001C010EC10922F1EC90101969093311E0E
:105320008093301E255D354FD9011C93CDCF83E08E
:105330000E9461052ECC903579F480EC90E00E94BB
:10534000620480E590E00E94620481E090E00E94A7
:1053500062048EE190E014CF983459F480EC90E030
:105360000E94620488E490E00E94620480E990E078
:1053700007CF993459F480EC90E00E94620489E4EC
:1053800090E00E94620482E990E0FACE973459F4EA
:1053900080EC90E00E94620487E490E00E94620446
:1053A00082E390E0EDCE933509F093C08091521ED8
:1053B000882309F489C08091571E882309F484C08A
:1053C0006091210A84ED9FE00E941B2160911402EC
:1053D00085ED9FE00E941B216091160286ED9FE003
:1053E0000E941B216091230A7091240A8091250A52
:1053F0009091260A692F77278827992787ED9FE0C4
:105400000E941B216091230A7091240A8091250A31
:105410009091260ABC018827992788ED9FE00E9479
:105420001B216091230A7091240A8091250A909192
:10543000260A672F782F892F992789ED9FE00E94F0
:105440001B216091230A8AED9FE00E941B2160913D
:10545000270A7091280A8091290A90912A0A692FB7
:105460007727882799278BED9FE00E941B21609169
:10547000270A7091280A8091290A90912A0ABC0172
:10548000882799278CED9FE00E941B216091270AB5
:105490007091280A8091290A90912A0A672F782F03
:1054A000892F99278DED9FE00E941B216091270A8B
:1054B0008EED9FE00E941B2163E78FED9FE00E942D
:1054C0001B218AE090E063CE8AE090E00E94FF0515
:1054D00060CB943509F05DCB60E08FED9FE00CCFA1
:1054E0001092491E0E94870402CA103C09F051CB59
:1054F000F092481EE09219021092311E1092301E56
:1055000048CB8F929F92AF92BF92CF92DF92EF9251
:10551000FF92CF93DF93EC01688179818A819B812F
:10552000611571058105910521F464E279ED8BE542
:1055300097E02DE133EF41E050E00E945F2C4901FC
:105540005A019B01AC01A7EAB1E40E947E2C6B01D9
:105550007C01ACEEB4EFA50194010E948C2CC60E28
:10556000D71EE81EF91EF7FE06C081E0C81AD10852
:10557000E10880E8F80AC882D982EA82FB82C70182
:10558000B6019F77DF91CF91FF90EF90DF90CF90A2
:10559000BF90AF909F908F9008958F929F92AF92FF
:1055A000BF92CF92DF92EF92FF9260911A027091B8
:1055B0001B0280911C0290911D02611571058105ED
:1055C000910521F464E279ED8BE597E02DE133EF6D
:1055D00041E050E00E945F2C49015A019B01AC015F
:1055E000A7EAB1E40E947E2C6B017C01ACEEB4EF23
:1055F000A50194010E948C2CC60ED71EE81EF91E30
:10560000F7FE06C081E0C81AD108E10880E8F80A70
:10561000C0921A02D0921B02E0921C02F0921D026C
:10562000C701B6019F77FF90EF90DF90CF90BF90BA
:10563000AF909F908F90089560931A0270931B0211
:1056400080931C0290931D0208950E94672B08F41A
:1056500081E00895E89409C097FB3EF49095809509
:10566000709561957F4F8F4F9F4F9923A9F0F92F28
:1056700096E9BB279395F695879577956795B795A6
:10568000F111F8CFFAF4BB0F11F460FF1BC06F5F8C
:105690007F4F8F4F9F4F16C0882311F096E911C09E
:1056A000772321F09EE8872F762F05C0662371F0BF
:1056B00096E8862F70E060E02AF09A95660F771FD3
:1056C000881FDAF7880F9695879597F90895990FAF
:1056D0000008550FAA0BE0E8FEEF16161706E807BC
:1056E000F907C0F012161306E407F50798F0621BDD
:1056F000730B840B950B39F40A2661F0232B242BB2
:10570000252B21F408950A2609F4A140A6958FEFD0
:10571000811D811D08950E949E2B0C940F2C0E94C8
:10572000012C38F00E94082C20F0952311F00C94E5
:10573000F82B0C94FE2B11240C94432C0E94202C4B
:1057400070F3959FC1F3950F50E0551F629FF001D4
:10575000729FBB27F00DB11D639FAA27F00DB11DED
:10576000AA1F649F6627B00DA11D661F829F222776
:10577000B00DA11D621F739FB00DA11D621F839FFD
:10578000A00D611D221F749F3327A00D611D231FD3
:10579000849F600D211D822F762F6A2F11249F5721
:1057A00050409AF0F1F088234AF0EE0FFF1FBB1F24
:1057B000661F771F881F91505040A9F79E3F5105E3
:1057C00080F00C94F82B0C94432C5F3FE4F3983E4C
:1057D000D4F3869577956795B795F795E7959F5F8D
:1057E000C1F7FE2B880F911D9695879597F908951F
:1057F00097F99F6780E870E060E008959FEF80EC84
:10580000089500240A941616170618060906089526
:1058100000240A9412161306140605060895092E8C
:105820000394000C11F4882352F0BB0F40F4BF2BFB
:1058300011F460FF04C06F5F7F4F8F4F9F4F08953B
:1058400057FD9058440F551F59F05F3F71F0479531
:10585000880F97FB991F61F09F3F79F08795089516
:10586000121613061406551FF2CF4695F1DF08C035
:10587000161617061806991FF1CF86957105610552
:1058800008940895E894BB2766277727CB0197F9FA
:105890000895F999FECF92BD81BDF89A992780B5F8
:1058A0000895262FF999FECF1FBA92BD81BD20BD64
:1058B0000FB6F894FA9AF99A0FBE01960895052E3C
:1058C00097FB1EF400940E94762C57FD07D00E948F
:1058D000912C07FC03D04EF40C94762C50954095F7
:1058E000309521953F4F4F4F5F4F0895909580958C
:1058F000709561957F4F8F4F9F4F08950E94B32CF5
:10590000A59F900DB49F900DA49F800D911D112413
:105910000895B7FF0C947E2C0E947E2C821B930B63
:105920000895A1E21A2EAA1BBB1BFD010DC0AA1FE0
:10593000BB1FEE1FFF1FA217B307E407F50720F0F8
:10594000A21BB30BE40BF50B661F771F881F991F73
:105950001A9469F760957095809590959B01AC01BC
:10596000BD01CF010895A29FB001B39FC001A39FC5
:10597000700D811D1124911DB29F700D811D112488
:10598000911D08950E94C92C6894B1110C94432C68
:1059900008950E94282C88F09F5798F0B92F9927D6
:1059A000B751B0F0E1F0660F771F881F991F1AF00A
:1059B000BA95C9F714C0B13091F00E94422CB1E001
:1059C00008950C94422C672F782F8827B85F39F000
:1059D000B93FCCF3869577956795B395D9F73EF4A3
:1059E00090958095709561957F4F8F4F9F4F08954B
:1059F000AA1BBB1B51E107C0AA1FBB1FA617B707F5
:105A000010F0A61BB70B881F991F5A95A9F7809510
:105A10009095BC01CD010895EE0FFF1F881F8BBF2D
:105A20000790F691E02D1994692796276927782722
:105A3000872778270895E894DF93CF93FC01DB0153
:105A40000E94B32C7F936F93E9019A01AC01BF933D
:105A5000AF933F932F93DF010E94B32C26F46C1B6E
:105A60007D0B820B930B9E01EB01FC010E94DB2D51
:105A7000AF91BF912F913F910E94DB2DBE01CF01CD
:105A8000F9012F913F91CF91DF910895689401C062
:105A9000E8948F929F92CF93DF930E94542DDF91D1
:105AA000CF919F908F90089588249924F401E40168
:105AB000B0E49F93AA279A158B049C04ED05FE057C
:105AC000CF05D007A10798F4AD2FDC2FCF2FFE2FE5
:105AD000E92D982C892E982F872F762F652F542FFC
:105AE000432F322F2227B85031F7BF9127C01B2EEA
:105AF000BF91BB27220F331F441F551F661F771FFF
:105B0000881F991F881C991CEE1FFF1FCC1FDD1FCB
:105B1000AA1FBB1F8A149B04EC05FD05CE05DF05FB
:105B2000A007B10748F08A189B08EC09FD09CE09C7
:105B3000DF09A00BB10B21601A94E1F62EF4940159
:105B4000AF01BE01CD01000C0895002E083090F089
:105B5000982F872F762F652F542F432F322F2227F0
:105B60000850F4CF220F331F441F551F661F771FA5
:105B7000881F991F0A95B2F7002D089597FD10947C
:105B8000002E083098F00850232F342F452F562F21
:105B9000672F782F892F912DF4CF1594979587959E
:105BA0007795679557954795379527950A95AAF75D
:105BB0001124002D08950E94B32C460F571FC81FB3
:105BC000D91F08F4319608950F931F93CF93DF9355
:105BD0008230910510F482E090E0E0911F1FF09177
:105BE000201F30E020E0B0E0A0E0309799F42115CC
:105BF000310509F44AC0281B390B24303105D8F58A
:105C00008A819B816115710589F1FB0193838283F0
:105C1000FE0111C04081518102811381481759074B
:105C2000E0F04817590799F4109761F012960C9319
:105C3000129713961C933296CF01DF91CF911F914B
:105C40000F91089500931F1F1093201FF4CF21156B
:105C5000310551F04217530738F0A901DB019A01D1
:105C6000BD01DF01F801C1CFEF01F9CF9093201FF3
:105C700080931F1FCDCFFE01E20FF31F81939193FD
:105C80002250310939832883D7CF20911D1F3091AD
:105C90001E1F232B41F420912002309121023093CA
:105CA0001E1F20931D1F20911E0230911F022115DF
:105CB000310541F42DB73EB74091220250912302A5
:105CC000241B350BE0911D1FF0911E1FE217F307F7
:105CD000A0F42E1B3F0B2817390778F0AC014E5F5C
:105CE0005F4F2417350748F04E0F5F1F50931E1F5C
:105CF00040931D1F819391939FCFF0E0E0E09CCFF4
:105D0000CF93DF930097E9F0FC0132971382128260
:105D1000A0911F1FB091201FED0130E020E01097EF
:105D2000A1F420813181820F931F20911D1F30919A
:105D30001E1F2817390709F061C0F0931E1FE0935A
:105D40001D1FDF91CF910895EA01CE17DF07E8F517
:105D50004A815B819E0141155105B1F7E901FB8341
:105D6000EA8349915991C40FD51FEC17FD0761F4DF
:105D7000808191810296840F951FE9019983888320
:105D8000828193819B838A83F0E0E0E012968D917B
:105D90009C9113970097B9F52D913C911197CD01E6
:105DA0000296820F931F20911D1F30911E1F2817EE
:105DB000390739F6309751F51092201F10921F1FA6
:105DC000B0931E1FA0931D1FBCCFD383C2834081FD
:105DD0005181840F951FC817D90761F44E5F5F4F3B
:105DE00088819981480F591F518340838A819B8103
:105DF000938382832115310509F0B0CFF093201FE2
:105E0000E0931F1F9ECFFD01DC01C0CF13821282E1
:065E1000D7CFF894FFCF8C
:105E1600FFDCFE7E037E037E037E037E037E037E1F
:105E2600037E03010500FF0011FE010000000000D3
:105E3600221F8000781E00A02800F03C0040510080
:105E4600127A00E4A20024F40048E80190D003206E
:105E5600A1070000000015047F03AC036704DD03FF
:105E6600BB03CF03000000006D1C321C831C381BD3
:105E7600241C5F1B391B4572726F722C20696E647D
:105E8600657465726D696E61746520626F6F7420EA
:105E9600766563746F720D0A004572726F722C20FC
:105EA600696E636F727265637420626F6F742076B9
:085EB6006563746F720D0A00B0
:00000001FF
